:020000040000FA
:0400000000001329C0
:08000800A000030E8312A10009
:100010000A08A2000408A3008C1C8A288C10A71DC3
:100020001928E10A0319E00A031D1928A71127104E
:100030000712B71B28284208B9070318B80A031982
:10004000B70A4108B8070318B70A4008B7073528A8
:1000500003104508B9070318B80A0319B70A44087A
:10006000B8070318B70A4308B7073F08BC073E089C
:1000700003183E0FBB073D0803183D0FBA070318CE
:10008000A714BA1F8715BA1B871100308A005908B8
:1000900082073B2A3D2A3F2A452A4B2A512A562AC3
:1000A0005A2ADC01DD0103105A18DC07DC0CDD0CD8
:1000B000DA18DC07DC0CDD0C5A19DC07DC0CDD0C73
:1000C000DA19DC07DC0CDD0C5A1ADC07DC0CDD0C61
:1000D000DA1ADC07DC0CDD0C5A1BDC07DC0CDD0C4F
:1000E000DA1BDC07DC0CDD0C5A09DE00DF01031033
:1000F000DE0CDF0C5F08DD070318DC0A5E08DC0796
:100100005D0D9516031C95125D0D1516031C151239
:100110005C0893002308840022088A00210E8300D3
:10012000A00E200E09000630A400A40B95289F14F1
:100130009F1898281E08AD0008008030E2000030AB
:10014000E3000030E400E601E7011830E500640D4B
:10015000E30DE20DE70DE60DE40D6108E70260082E
:10016000031C600FE602031864146418BA28E6073B
:100170006108E707E50BA7280800E801E901EA01A3
:10018000550803104718E807E80CE90CEA0CC718F3
:10019000E807E80CE90CEA0C4719E807E80CE90C59
:1001A000EA0CC719E807E80CE90CEA0C471AE8075B
:1001B000E80CE90CEA0CC71AE807E80CE90CEA0CB1
:1001C000471BE807E80CE90CEA0CC71BE807E80C3A
:1001D000E90CEA0C4618E807E80CE90CEA0CC6182A
:1001E000E807E80CE90CEA0C4619E807E80CE90C0A
:1001F000EA0CC619E807E80CE90CEA0C461AE8070D
:10020000E80CE90CEA0CC61AE807E80CE90CEA0C61
:10021000461BE807E80CE90CEA0CC61BE807E80CEB
:10022000E90CEA0C080087010730990091010430BD
:10023000920093018C01C0308B000C309500831626
:1002400002308C003730910020309F00FF30920048
:100250003F30850007308700D330810083120230A1
:10026000D500D700D800FF30DA008030C800D901AF
:10027000A701AE01AF01B0015430B100B901B8011E
:10028000B7010330BD00BE00BF000330C600C70089
:10029000C001C101C201C301C401C501AC012908EB
:1002A000A806A90905080839A40007080439240488
:1002B0002A06A905A805FF3A28042904FF3AAA0638
:1002C000AB002B1D75292A197529D80A5808063A3A
:1002D0000319D80158087A22D500BD206808BD004E
:1002E0006908BE006A08BF000A2AAB1D9F29AA1927
:1002F0009F2927188829E001E101A715071627146F
:10030000B701B801B901BA01BB01BC01A7149F290B
:10031000A711071227109D206308C6006408C700B4
:10032000BD206808BD006908BE006A08BF00271527
:1003300004305207D300D3090930D4000A2AAC0A8A
:1003400001308A002C0807398207AD29C429D52934
:10035000F529FB290730AC004F2901309F0093207D
:10036000D200271DB8295307540703184F29271116
:100370009A24C600A125C700BD206808BD006908F1
:10038000BE006A08BF000A2A05309F009320043E81
:10039000E039A4002D08E0392406031D4F29AD0ED5
:1003A000AD0C07302D05D9004F2909309F0093204F
:1003B000043EE039A4002D08E0392406031D4F292E
:1003C000AD0EAD0C07302D05A400570203194F29BF
:1003D0002408D700D8007A22D500BD206808BD00C7
:1003E0006908BE006A08BF000A2A11309F009320E6
:1003F0002D08DA004F2915309F009320FC39031D8A
:10040000032A0430082AFF3AFC3903190330FF3A63
:10041000C8000A2AD10103103E0CCF003F0CD000C7
:10042000D10C4808CD0024224908C0004A08C10068
:100430004B08C2004809CD0024224908C3004A08DD
:10044000C4004B08C5004F29CC011830CE004F081E
:10045000C9005008CA005108CB004B0DCA0DC90D88
:10046000CC0DCB0D4D08CC0203184B144B1CCC0704
:10047000CE0B2D2A08003708512837095128B71B01
:10048000432A00305128FF3051280310380D370D12
:10049000B71FFF3A5128380D370DB71BFF3A8A2294
:1004A000512837089223FF3AA50051283708922394
:1004B000A50051282E08A71C5128A7103108B50007
:1004C000B600B2003008B300B400B30DB50DB30DE3
:1004D000350DB206B60CB40C3408B206B60C340CAA
:1004E000B2063008B1002F08B0002E08AF00320865
:1004F000AE005128A50002308A002508823E03186C
:100500008A0A820001340234033404340634083485
:1005100002340234A50002308A002508923E0318F6
:100520008A0A8200FF34FF34FF34FF34FF34FF3483
:10053000FF34FE34FE34FE34FE34FE34FE34FD342B
:10054000FD34FD34FC34FC34FC34FB34FB34FB342C
:10055000FA34FA34F934F934F834F834F734F73437
:10056000F634F634F534F434F434F334F234F2344B
:10057000F134F034F034EF34EE34ED34ED34EC3467
:10058000EB34EA34E934E834E734E634E634E5348D
:10059000E434E334E234E134E034DF34DE34DD34B7
:1005A000DB34DA34D934D834D734D634D534D434EF
:1005B000D234D134D034CF34CE34CC34CB34CA342A
:1005C000C834C734C634C534C334C234C134BF346C
:1005D000BE34BD34BB34BA34B834B734B634B434B2
:1005E000B334B134B034AE34AD34AC34AA34A934FD
:1005F000A734A634A434A334A134A0349E349D344B
:100600009B349A349834963495349334923490349D
:100610008F348D348C348A348934873485348434EF
:10062000823481347F347E347C347B347934773443
:10063000763474347334713470346E346D346B3496
:100640006A346834663465346334623460345F34E9
:100650005D345C345A34593457345634543453343A
:10066000523450344F344D344C344A344934483485
:10067000463445344334423441343F343E343D34CF
:100680003B343A3439343834363435343434323413
:10069000313430342F342E342C342B342A34293452
:1006A000283427342634253423342234213420348A
:1006B0001F341E341D341C341B341A341A341934BC
:1006C00018341734163415341434133413341234E4
:1006D0001134103410340F340E340E340D340C3405
:1006E0000C340B340A340A3409340934083408341D
:1006F000073407340634063405340534053404342D
:100700000434043403340334033402340234023432
:10071000023402340234013401340134013401342E
:1007200001340134A50003308A0025089A3E0318DD
:100730008A0A8200FF34FF34FF34FF34FF34FF3471
:10074000FE34FE34FE34FD34FD34FD34FC34FC3420
:10075000FB34FB34FA34F934F934F834F734F73431
:10076000F634F534F434F334F234F134F034EF3455
:10077000EE34ED34EC34EA34E934E834E634E5348C
:10078000E434E234E134DF34DE34DC34DB34D934D5
:10079000D734D634D434D234D034CF34CD34CB342F
:1007A000C934C734C534C334C134BF34BD34BB3499
:1007B000B934B634B434B234B034AD34AB34A93413
:1007C000A634A434A2349F349D349A34983495349A
:1007D000933490348E348B3488348634833480342C
:1007E0007E347B3478347534733470346D346A34C9
:1007F0006734643462345F345C345934563453346F
:1008000050344D344A344734443441343E343B341C
:100810003834353432342F342B34283425342234D0
:100820001F341C3419341634133410340C34093486
:100830000634033400340334063409340D341034E0
:100840001334163419341C341F342234253429341B
:100850002C342F343234353438343B343E34413444
:10086000443447344A344D34503453345634593474
:100870005C345F346234643467346A346D347034A9
:100880007334753478347B347E34803483348634E6
:1008900088348B348E3490349334953498349A342D
:1008A0009D349F34A234A434A734A934AB34AE347D
:1008B000B034B234B434B734B934BB34BD34BF34DB
:1008C000C134C334C534C734C934CB34CD34CF3448
:1008D000D134D234D434D634D734D934DB34DC34C4
:1008E000DE34DF34E134E234E434E534E734E83450
:1008F000E934EA34EC34ED34EE34EF34F034F134EE
:10090000F234F334F434F534F634F734F734F8349D
:10091000F934F934FA34FB34FB34FC34FC34FD3460
:10092000FD34FD34FE34FE34FE34FF34FF34FF3436
:10093000FF34FF3404308A002D08A13E03188A0AD0
:1009400082000034003400340034003400340034B9
:1009500000340034003400340034003400340034F7
:1009600000340034003400340034003400340034E7
:1009700000340034003400340034003400340034D7
:1009800000340034003400340034003400340034C7
:1009900000340034003400340034003400340034B7
:1009A00000340034003400340034003400340034A7
:1009B0000034003400340034003400340034003497
:1009C0000034003400340034003400340034003487
:1009D0000034003400340034003400340034003477
:1009E0000034003400340034003400340034003467
:1009F0000034003400340034003400340034003457
:100A00000034003400340034003400340034003446
:100A10000034003400340034003400340034003436
:100A20000034003400340034013401340134013422
:100A3000013401340134013401340134013401340E
:100A400001340134013401340134013401340134FE
:100A500001340134013401340134013401340134EE
:100A600001340134013401340234023402340234DA
:100A700002340234023402340234023402340234C6
:100A800002340234023402340234023402340334B5
:100A9000033403340334033403340334033403349E
:100AA000033403340334033404340434043404348A
:100AB0000434043404340434043404340534053474
:100AC000053405340534053405340534053406345D
:100AD0000634063406340634063406340734073444
:100AE000073407340734073408340834083408342A
:100AF0000834093409340934093409340A340A340D
:100B00000A340A340A340B340B340B340B340C34EF
:100B10000C340C340D340D340D340D340E340E34CD
:100B20000E340F340F340F341034103410341134A9
:100B30001134123412341234133413341434143480
:100B4000153405308A002D08A83E03188A0A820051
:100B5000163416341634173417341834183419343C
:100B60001A341A341B341B341C341D341D341E3407
:100B70001E341F34203420342134223423342334CF
:100B800024342534263427342734283429342A348D
:100B90002B342C342D342E342F3430343134323441
:100BA0003334343435343734383439343A343C34EB
:100BB0003D343E3440344134423444344534473487
:100BC00048344A344C344D344F3451345234543414
:100BD000563458345A345C345E346034623464348D
:100BE000663469346B346D347034723475347734F0
:100BF0007A347C347F348234853488348B348E3438
:100C00009134943497349A349E34A134A534A83462
:100C1000AC34B034B434B834BC34C034C434C83464
:100C2000CD34D134D634DA34DF34E434E934EE343C
:100C3000F334F934FE34043409340F3415341B34DE
:100C4000213428342E3435343C3442344A3451343F
:100C50005834603467346F34773480348834903457
:100C60009934A234AB34B534BE34C834D234DC3415
:100C7000E734F134FC34073413341E342A34363468
:100C800043344F345C346A34773485349334A2343B
:100C9000B034BF34CF34DF34EF34FF341034213478
:100CA00033344434573469347D349034A434B93403
:100CB000CD34E334F8340F3425343D3454346D34BA
:100CC00086349F34B934D334EE340A342634433472
:100CD00061347F349E34BD34DD34FE3420344234FC
:100CE00065348934AE34D334F93420344834713423
:100CF0009B34C534F1341E344B347934A934DA349E
:100D00000B343E347234A734DD3414344C3486341E
:100D1000C134FD343B347A34BA34FC343F34843447
:100D2000CA3412345B34A634F23441349134E234A0
:100D300036348B34E2343B349634F3345234B334A7
:100D400016347C34E3344D34B934283499340C34BB
:02400E00C230BE
:00000001FF
